S01800006275696C642F6D696361322F6D61696E2E737265632D
S11300000C945F010C947C010C947C010C947C0195
S11300100C947C010C947C010C947C010C947C0168
S11300200C947C010C947C010C947C010C947C0158
S11300300C947C010C947C010C947C010C94D40BE6
S11300400C947C010C947E010C9406020C947C01AB
S11300500C9430020C9410080C947C010C947C01D8
S11300600C947C010C947C010C947C010C947C0118
S11300700C947C010C947C010C947C010C947C0108
S11300800C947C010C947C010C947C01001C005E9B
S113009000FA017301EA04BC0A5E050202020202CC
S11300A002000000140055008700B901E5043D007A
S11300B0080808080808AEEFEFEFEFEFEF000021A3
S11300C010422063308440A550C660E7700881293F
S11300D0914AA16BB18CC1ADD1CEE1EFF1311210D7
S11300E00273325222B5529442F772D6623993188F
S11300F0837BB35AA3BDD39CC3FFF3DEE3622443E3
S11301003420040114E664C774A44485546AA54BDE
S1130110B528850995EEE5CFF5ACC58DD553367276
S11301202611163006D776F6669556B4465BB77A2E
S1130130A719973887DFF7FEE79DD7BCC7C448E502
S1130140588668A7784008611802282338CCC9ED7E
S1130150D98EE9AFF9488969990AA92BB9F55AD416
S11301604AB77A966A711A500A333A122AFDDBDCCE
S1130170CBBFFB9EEB799B588B3BBB1AABA66C8722
S11301807CE44CC55C222C033C600C411CAEED8F1E
S1130190FDECCDCDDD2AAD0BBD688D499D977EB6B6
S11301A06ED55EF44E133E322E511E700E9FFFBE6E
S11301B0EFDDDFFCCF1BBF3AAF599F788F8891A941
S11301C081CAB1EBA10CD12DC14EF16FE18010A118
S11301D000C230E3200450254046706760B983981C
S11301E093FBA3DAB33DC31CD37FE35EF3B1029068
S11301F012F322D2323542145277625672EAB5CBE8
S1130200A5A89589856EF54FE52CD50DC5E234C3B7
S113021024A01481046674476424540544DBA7FABB
S1130220B79987B8975FE77EF71DC73CD7D326F207
S1130230369106B01657667676154634564CD96D07
S1130240C90EF92FE9C899E9898AB9ABA944586557
S11302504806782768C018E1088238A3287DCB5C5B
S1130260DB3FEB1EFBF98BD89BBBAB9ABB754A54A7
S11302705A376A167AF10AD01AB32A923A2EFD0F27
S1130280ED6CDD4DCDAABD8BADE89DC98D267C07F7
S11302906C645C454CA23C832CE01CC10C1FEF3EFB
S11302A0FF5DCF7CDF9BAFBABFD98FF89F176E3647
S11302B07E554E745E932EB23ED10EF01E00112474
S11302C01FBECFEFD0E1DEBFCDBF11E0A0E0B1E0B3
S11302D0EAE2F5E200E00BBF02C007900D92AC34F5
S11302E0B107D9F712E0ACE4B1E001C01D92A43C1F
S11302F0B107E1F70C947D020C9400001F920F9259
S11303000FB60F9211242F933F934F935F936F93E4
S11303107F938F939F93AF93BF93EF93FF939FB17B
S1130320809103028FB9892F0E94D108FF91EF9128
S1130330BF91AF919F918F917F916F915F914F91F9
S11303403F912F910F900FBE0F901F901895AF9271
S1130350BF92CF92DF92EF92FF920F931F93CF93AE
S1130360DF9386EEF82EA090B402B090B502C09050
S1130370B602D090B702A114B104C104D10481F132
S1130380EE246AE572E000E010E081E090E0002EE7
S113039002C0880F991F0A94E2F7AA2797FDA09537
S11303A0BA2F8A219B21AC21BD210097A105B1055B
S11303B079F02F2D332744275527FB01858196811A
S11303C0A781B08582179307A407B5070CF4F580BD
S11303D0E3940F5F1F4F675F7F4FF1E0FE15A8F6B0
S11303E08FB7F8949927F0927F02F1BE10927402AD
S11303F08FBF0E944B07DF91CF911F910F91FF9008
S1130400EF90DF90CF90BF90AF9008951F920F921E
S11304100FB60F9211242F933F934F935F936F93D3
S11304207F938F939F93AF93BF93EF93FF935F9BC0
S113043006C08CB140E050E060E00E94110CFF91D6
S1130440EF91BF91AF919F918F917F916F915F9148
S11304504F913F912F910F900FBE0F901F901895C1
S113046078941F920F920FB60F9211242F933F93FB
S11304704F935F936F937F938F939F93AF93BF93A8
S1130480EF93FF930E948A0EFF91EF91BF91AF917A
S11304909F918F917F916F915F914F913F912F9198
S11304A00F900FBE0F901F901895AC018FB7F89462
S11304B0282F3327E0917102809171028F5F80931E
S11304C07102809171028770809371029091710220
S11304D080912502981759F02FBFFF27EE0FFF1FB9
S11304E0E451FE4F4083518381E090E00895E0930E
S11304F071022FBF80E090E00895C5EED0E1DEBF29
S1130500CDBFD29AD09AD19AD698A79AA69AA59AEC
S1130510A49AA39AA29AA19AA09A8C9A8F9A8E9A34
S1130520BB98BF98D498DC98D39A8B9A8D9ADB9A0F
S1130530DA9AD89AD99A83E08C5F8739E8F310E085
S11305408AE08093B20110937102109325028CEB20
S113055091E09093AA028093A9021093AE010E94A5
S113056047060E9476068FB7F8949927109376026F
S11305708FBF8FB7F894282F332781E08093AF0182
S1130580880F80934C018AE292E0909373028093E7
S1130590720210932E0282E290E090936D02809397
S11305A06C021093E9011092BD021092BC021092E9
S11305B0BB011092BA011092FE011092FD0110933A
S11305C0AC011093A90110938F028FEF9FEF9093CA
S11305D078028093770290937A0280937902109341
S11305E0590210937D02E6EBF0E0849199279093F1
S11305F05602809355022FBF8FB7F8949927B99864
S1130600BB98BA986B986A986F9A6E9A8FBFD6986F
S11306108C9A8E9A8F9A949A979A969A6AE3812FD3
S11306200E94BA066BE3812F0E94BA0680ED97E020
S113063000000000000000000000000000000000B6
S1130640019718161906A4F380E880930F02682F07
S11306508BE00E94BA0680E980931102682F84E03F
S11306600E94BA06109213028FE68093140285E565
S113067080931502609113028FE00E94BA06809164
S11306801402682F80E10E94BA0680911502682F37
S113069081E10E94BA0611E010931702612F83E1F1
S11306A00E94BA061093220219821A821B821C82AB
S11306B020E030E040E050E02D833E834F835887B4
S11306C0BA01A90149875A876B877C876FEF7FEF4F
S11306D08FEF9FE76D877E878F87988B198A1A8A99
S11306E01B8A7B897C8B83E091E08D8B9E8BA7E2B8
S11306F0B1E0AF8BB88FE0E0F0E0E98FFA8FAD891D
S1130700BE89AD90BD90CD90DD90AD8BBE8BEE24B7
S1130710FF2487011701280160E070E885E497E66B
S1130720A60195010E947312DA01C90181709070CB
S1130730A070B070892B21F02F5F3F4F4F4F5F4F58
S113074021FF0BC0212CA0E23A2E412C512C860112
S1130750750116950795F794E794E2E05695479549
S113076037952795EA95D1F7DA01C9017EE0880F1C
S1130770991FAA1FBB1F7A95D1F7820D931DA41D43
S1130780B51D212C60EE362E6FEF462E6FEF562EE0
S1130790280E391E4A1E5B1E80509042A044B04071
S11307A080509C49AF4BB04008F060C0AF89B88D11
S11307B08D919C91AA27BB2742013101681A790ABD
S11307C08A0A9B0AD401C30180509040A044B040DF
S11307D080509C49AF4BB04008F048C0CA01B901F1
S11307E0A60195010E945412DC01CB01E80EF91E0A
S11307F00A1F1B1F20E136EB4DEF5FEFE20EF31EE5
S1130800041F151FD801C70180519641AF4CB9414F
S1130810B7FF07C0B095A095909581959F4FAF4FB6
S1130820BF4F4D855E856F85788984179507A60728
S1130830B707E4F42D823E824F82588669867A8611
S11308408B869C86E982FA820B831C83298D3A8DE0
S1130850275C3E4FF90120813181298B3A8BFC8939
S1130860FA5FFB8B8D879E87AF87B88B2C892F5FB0
S11308702C8B498D5A8D4E5F5F4F498F5A8F6F89EC
S1130880788D6E5F7F4F6F8B788F293008F437CF68
S11308907B89772309F460C08D81809307022D81C1
S11308A03E814F815885BB27A52F942F832F80939A
S11308B00602CA01AA27BB27809305023985309313
S11308C00A0249855A856B857C85BB27A72F962FFD
S11308D0852F80930902CB01AA27BB2780930802A6
S11308E0598950930C0269897A89872F99278093B3
S11308F00B0289819A81AB81BC818030E5E69E0739
S1130900EDECAE07EDE1BE07A8F480509448A74D86
S1130910B74128F484E880930D0281E904C084E49B
S113092080930D0281E88093210282E080930E027D
S113093080E70AC08CE880930D0283EF8093210244
S113094082E380930E0280E2809316022B89220FA9
S1130950220F220F2093100249815A816B817C81DE
S11309604093B8025093B9026093BA027093BB02E9
S113097011E065E0E62E62E0F62ED7018D917D014F
S1130980682F812F0E94BA061F5F1D30B0F380913B
S11309901602682F82E10E94BA0660E08BE00E9492
S11309A0BA066FE382E40E94BA0661E180E00E9425
S11309B0BA0666EA8EE00E94BA068EE00E94DE065F
S11309C083FFFBCF66E28EE00E94BA0661EE80E010
S11309D00E94BA0680912102682F89E00E94BA061B
S11309E060E08BE00E94BA0666EA8EE00E94BA06D6
S11309F01EE0812F0E94DE0683FFFACF66E2812F7C
S1130A000E94BA0680E980931102682F8DE00E944B
S1130A10BA0680912202282F33278FB7F89499279A
S1130A202093A7028FBF0E9411078FB7F8949927CC
S1130A30109299028FBF8FB7F89499271092C3022E
S1130A401092C202109298021092970210922902F8
S1130A50109228028FBF0E9411078FB7F89499272C
S1130A6016B917B88FBF8FB7F894482F5527209120
S1130A7000013091010181E597E3289FF001299F4E
S1130A80F00D389FF00D1124CF018F5A984C90939C
S1130A908D0280938C029093C0028093BF0285E8FC
S1130AA09FE0289FB001299F700D389F700D11247D
S1130AB0CB018B57904F9093B4018093B3014FBFF8
S1130AC00E94470680910001909101019093B10228
S1130AD08093B0021092B3021092AE021092AD0253
S1130AE01092580210925702AA980E947606109209
S1130AF090008FE089B922E02BB966E060939500FD
S1130B0088ED8AB98FB7F89499277091AF018FBF98
S1130B10713009F07EC08FB7F894482F5527E091C3
S1130B207202F091730214822093AF011092A90112
S1130B301092AC018FEF9FEF90937802809377022D
S1130B40809159029927880F991FFC01E457FF4FA0
S1130B5024913327322F222783579F4FFC018491FE
S1130B609927282B392B3093B9012093B8014FBF13
S1130B7080917D02882369F56BE30E94BA0680EDBB
S1130B8097E00000000000000000000000000000EA
S1130B900000019718161906A4F369E380E00E9487
S1130BA0BA0688EC90E0000000000000000000009D
S1130BB0000000000000019718161906A4F3BB9862
S1130BC0BA980E942C0780EC8DB9B8980E944B0704
S1130BD020C09927880F991FFC01EF55FF4F2491DE
S1130BE03327322F22278E559F4FFC01849199275A
S1130BF0282B392B8FB7F89499276093AF018FBFB7
S1130C00C901AA27BB279C01AD01672F872F0E942A
S1130C105D0728EE33E040E050E060E0862F0E945C
S1130C205D071092B3020E944B07789490912502BD
S1130C3080917102981719F480E090E01FC08FB77B
S1130C40F894282F332790912502809125028F5FF5
S1130C508093250280912502877080932502E92FD5
S1130C60FF27EE0FFF1FE451FE4F80819181108218
S1130C7011822FBFFC01099581E090E08823B1F631
S1130C8085B7806285BF889500000000CFCF1092A1
S1130C90B4021092B5021092B6021092B7021092EA
S1130CA074028FEF8093BE028093A7011092EA0131
S1130CB083E08093750296EE90937F028FB7F89449
S1130CC0282F332787B78E7F87BF87B78D7F87BF4E
S1130CD080B7886080BF8BE083BF12BE91BF87B7A7
S1130CE0826087BF2FBF81E090E008958FB7F894AA
S1130CF0682F80E090E04FE451E09C01F901E80F97
S1130D00F91FE058FD4F44835583128213821182E8
S1130D1001962B5F3F4F455D5F4F8230910574F321
S1130D201092A60210926F0210926E021092B101FC
S1130D301092B00110924E0110924D011092A60132
S1130D401092A5011092A50210927B021092A802A3
S1130D501092B7011092B601109200021092FF0196
S1130D6080918402909185029093920280939102E3
S1130D706FBF0895880F949896E087FF02C0979AF2
S1130D8001C097989698969A880F915097FFF5CF3F
S1130D90979A9698969A949A97E067FF02C0979AC2
S1130DA001C097989698969A660F915097FFF5CF41
S1130DB0949A979A969A81E090E0089590E0880F2B
S1130DC0949826E030E087FF02C0979A01C0979874
S1130DD09698969A880F2150304037FFF4CF27E039
S1130DE030E097989698969A8F98949A969840E0BF
S1130DF050E0879941E0892F9927215030404423BE
S1130E0029F0880F991F982F916002C0982F990F8D
S1130E10969A37FFEBCF949A8F9A979A892F9927AE
S1130E2008958FB7F894282F8091B501882391F401
S1130E3080E090E0E9E9F2E0819301968C3091053D
S1130E40DCF38EE18093A3028FE18093A40281E01E
S1130E508093B5012FBF089561E180E00E94BA0636
S1130E6080910D02682F89E00E94BA0660E08BE051
S1130E700E94BA068AEF90E0000000000000000023
S1130E800000000000000000019718161906A4F3E2
S1130E9081E090E0089580914B01882329F482ED4C
S1130EA090E10E94550206C085B7837E85BF85B751
S1130EB0806285BF80E090E00895CF92DF92EF9248
S1130EC0FF920F931F93CF93DF9379018A018230AE
S1130ED010F462301CF080E090E053C0282F3327D8
S1130EE0F90193E0EE0FFF1F9A95E1F7E20FF31F6C
S1130EF0E65AFD4FE182F2820383148360838FB745
S1130F00F894C82FDD2782B7E80EF11C011D111DCE
S1130F10E582F6820783108781E0C82ED12CC601B2
S1130F2002C0880F991F2A95E2F79C01442737FDD8
S1130F304095542F8091B4029091B502A091B602CD
S1130F40B091B702822B932BA42BB52B8093B402C0
S1130F509093B502A093B602B093B70280917F023A
S1130F609927AA27BB27E816F9060A071B0738F4AE
S1130F70E0927F02E1BE109274020E944B07CFBF41
S1130F80C601DF91CF911F910F91FF90EF90DF90F9
S1130F90CF9008950F931F93CF93DF93EC0120918B
S1130FA000013091010180915702909158020196FD
S1130FB090935802809357028AA19BA1019751F5FF
S1130FC09B8180910201981729F5888199814FEFBF
S1130FD08F3F940719F082179307E1F49A8183E015
S1130FE08C5F8B32E8F3983089F40091A902109158
S1130FF0AA0281E08093AE01D093AA02C093A90211
S11310008AE59FE00E945502C80101C0CE01009705
S113101009F0EC01CE01DF91CF911F910F9108955A
S11310201F920F920FB60F921124FF920F931F93EA
S11310302F933F934F935F936F937F938F939F93DC
S1131040AF93BF93CF93DF93EF93FF93C4B1D5B125
S1131050D370349A379878948FB7F894F82E809197
S1131060C202082F112721E030E0002E02C0220F17
S1131070331F0A94E2F78091970290919802822399
S11310809323892B61F420953095809128029091C7
S1131090290282239323909329028093280240916A
S11310A02802509129024115510511F12091C202E3
S11310B03091C3022F5F3F4F2C30310511F0C9012D
S11310C002C080E090E09C0181E090E0022E02C02A
S11310D0880F991F0A94E2F784239523892B51F3EF
S11310E03093C3022093C2028091C2020E94BF08BF
S11310F0FFBE0115110569F48FB7F894282F332723
S1131100D0937A02C093790281E080938F022FBF3B
S113111001C080E099272FB7F8948823C9F461E0CF
S113112070E002C0660F771F0A95E2F740919702BC
S113113050919802CA0186239723892B49F0CB0149
S11311408095909548235923509398024093970291
S11311502FBFFF91EF91DF91CF91BF91AF919F91FD
S11311608F917F916F915F914F913F912F911F913B
S11311700F91FF900F900FBE0F901F901895982F0E
S11311808FB7F894282F3327E9E9F2E0E90FF11D2E
S113119080818F7187B92FBF379A369A81E090E0AA
S11311A008951F93CF93682F8091A70281116095B2
S11311B08091AF01482F55274230510509F4ADC045
S11311C04330510524F44115510571F0B8C244303F
S11311D0510509F47EC1443051050CF404C1453075
S11311E0510509F4EEC1ABC2209193028FB7F89474
S11311F09927209303028FBF6091AB027091AC02D8
S11312006F5F7F4F7093AC026093AB0280914C018F
S113121099278430910559F18530910534F4823051
S1131220910559F00397B1F06AC08630910509F42D
S11312305EC006970CF44BC062C08091B8019091D7
S1131240B9016817790708F47AC283E3809393029B
S113125083E052C08CEC8093930284E080934C0131
S11312608FEF9FEF9093AC028093AB0268C28091A2
S1131270AB02282F33278091E7019091E8012817CA
S11312803907F8F4E0919502F0919602E60FF71F02
S11312902081209393028091010290910202EDEB50
S11312A0F0E02927220FF11DE20FF11DC895982FB8
S11312B0802D3196C8959025909302028093010267
S11312C03EC2809101028093930285E015C0809113
S11312D0010290910202892F99278093930286E05C
S11312E080934C015093AC024093AB0228C264300B
S11312F0710508F424C287E080934C0120C2BB9896
S1131300BA980E942C071092AC0180E190E10E94EF
S11313105502882309F413C2AFC16A3A11F0653546
S113132071F52091BC023091BD022F5F3F4F309385
S1131330BD022093BC0280917D02E82FFF27E65670
S1131340FF4F849199278217930708F0F8C11092F0
S1131350B2021092BD021092BC02109227021092A7
S113136026021092E901109202021092010282E216
S113137090E090936D0280936C0284E07EC1809132
S1131380AC01882309F4DBC1809177029091780243
S113139001979093780280937702181619060CF43B
S11313A0CEC110928F028FB7F894C82F20912802D3
S11313B03091290220FD10C0C90181609093290257
S11313C0809328022115310539F43093C302209308
S11313D0C20280E00E94BF08CFBF1092BD021092EB
S11313E0BC0283E04AC16A3A09F45EC0653509F477
S11313F05BC080918F02882309F4A1C180917D0292
S1131400E82FFF27EA54FF4F8491282F3327809138
S1131410790290917A022817390708F045C061EEE5
S113142080E00E94BA0680912102682F89E00E9420
S1131430BA068AEF90E000000000000000000000FF
S1131440000000000000019718161906A4F380910B
S11314500F02682F8BE00E94BA0684E190E000003E
S113146000000000000000000000000000000197E0
S113147018161906A4F3BB9ABA9A1092AC021092E9
S1131480AB0210920202109201021092AF0182E0AC
S113149080934C012AEA209393028FB7F8949927FA
S11314A0209303028FBF4BC10E94A90B8F709070D1
S11314B024E230E0829FA001839F500D929F500D43
S11314C01124CA01820F931F9093780280937702AC
S11314D0D3C06A3A11F0653519F46093FE012FC147
S11314E08091B2029927009721F003970CF060C015
S11314F003C06093FD015FC02091FD013091FE01A6
S1131500922F88279093FE018093FD016093FD0143
S113151010E0220F331F67FD2160660F53E32C3C5C
S1131520350709F040C0E0917202F09173024481E2
S11315304423B9F08FB7F894382F2091940220FFF8
S113154006C08FB7F8949927DA9A2E7F05C08FB713
S1131550F8949927DA982160209394028FBF3FBFB3
S113156027C085E08093AF018FB7F894C82F2091EE
S113157028023091290220FD10C0C9018160909396
S11315802902809328022115310539F43093C302CE
S11315902093C202842F0E94BF08CFBF87E0811B23
S11315A08093E90108C01F5F183008F4B2CF03C06C
S11315B082E08093AF018091B2028F5F8093B20288
S11315C0BEC08091FD019091FE01982F88279093D1
S11315D0FE018093FD016093FD012091FD01309196
S11315E0FE010090E90102C0369527950A94E2F7BE
S11315F0622FE0917202F091730280912602909121
S11316002702E80FF91F20834091260250912702F8
S11316104F5F5F4F509327024093260280916C02E4
S113162090916D024817590798F5809101029091A5
S11316300202EDEBF0E06927660FF11DE60FF11DE4
S1131640C895982F802D3196C895902590930202C5
S1131650809301024530510509F071C0E091720296
S1131660F09173028481992790936D0280936C02A8
S11316708E31910528F0148282E08093AF015FC01F
S11316800097F1F0059690936D0280936C0257C019
S113169048175907E1F48091010290910202EDEBA1
S11316A0F0E06927660FF11DE60FF11DC895982F2C
S11316B0802D3196C8959025909302028093010263
S11316C082E290E0909327028093260238C044324D
S11316D05105A8F1E0917202F091730222A133A1A5
S11316E080910102909102022817390729F481E0C0
S11316F090E082A393A302C012A213A20E94CC0B77
S1131700C2E0C093AF01E0917202F0917302809144
S1131710790290917A0284A395A38EEC9FE00E94B3
S11317205502882361F4E0917202F091730284837C
S1131730C093AF0180EC8DB9B8980E944B0781E04B
S113174090E0CF911F9108951092B30281E090E050
S113175008958FB7F894482F552720918C02309123
S11317608D02832F881F8827881F220F331F882309
S113177021F08BE090E1282739272F5F3F4F3093EA
S11317808D0220938C028091B3019091B40128279B
S113179039274FBFC90108956F98B89AC0980E941D
S11317A04B0781E090E0089578941F920F920FB652
S11317B00F9211242F933F934F935F936F937F93D3
S11317C08F939F93AF93BF93EF93FF938FB7F89447
S11317D0282F33278091EB01882369F080917002D0
S11317E08093900288608093700283BF8091FC0193
S11317F081BF1092EB012FBF85E290E10E94550258
S1131800FF91EF91BF91AF919F918F917F916F91D4
S11318105F914F913F912F910F900FBE0F901F90AA
S11318201895382F8091A50299278230910509F4E3
S11318306BC0833091052CF4009759F0019781F126
S1131840B7C18330910509F49CC0049709F459C1C8
S1131850AFC13E3709F0AEC180917B029927FC01EC
S1131860EE0FFF1FEE0FFF1FE80FF91FE80FF91F20
S1131870E058FD4F82819381009709F09BC111824A
S1131880909300028093FF019093B7018093B60177
S113189084819581909392028093910281E085C125
S11318A03E3709F487C180917B029927FC01EE0F32
S11318B0FF1FEE0FFF1FE80FF91FE80FF91FE05895
S11318C0FD4F30838091FF0190910002EDEBF0E039
S11318D0232F2927220FF11DE20FF11DC895982F00
S11318E0802D3196C8959025909300028093FF0136
S11318F0832F99278134910529F08234910509F4C5
S113190053C156C182E051C13E3709F451C16091BF
S11319107B023D3781F4862F9927FC01EE0FFF1FD0
S1131920EE0FFF1FE80FF91FE80FF91FE058FD4FF6
S113193080E281833FC1862F9927FC01EE0FFF1FB0
S1131940EE0FFF1FE80FF91FE80FF91FE058FD4FD6
S11319502181232721838091FF0190910002EDEBE7
S1131960F0E02927220FF11DE20FF11DC895982FF1
S1131970802D3196C8959025909300028093FF01A5
S113198013C14091B6015091B7014C32510508F092
S1131990BAC03D3711F484E008C13E3709F07FC076
S11319A04230510508F45FC0E0919102F091920237
S11319B0E40FF51F82919927382F222782919927C6
S11319C0282B392B8091FF019091000260917B02BA
S11319D028173907E1F4862F9927FC01EE0FFF1F22
S11319E0EE0FFF1FE80FF91FE80FF91FE058FD4F36
S11319F042505040428353838AE091E10E94550251
S1131A0080917B028F5F817080937B0210C0862F50
S1131A109927FC01EE0FFF1FEE0FFF1FE80FF91FC0
S1131A20E80FF91FE058FD4F128213821182809152
S1131A307B029927FC01EE0FFF1FEE0FFF1FE80F3B
S1131A40F91FE80FF91FE058FD4F82819381892B1C
S1131A50D9F484819581909392028093910281E0DC
S1131A608093A50213C080917B029927FC01EE0F9D
S1131A70FF1FEE0FFF1FE80FF91FE80FF91FE058D3
S1131A80FD4F1282138211821092A502109200025D
S1131A901092FF011092B7011092B6018BC0E09131
S1131AA09102F0919202E40FF51F30834091B60148
S1131AB05091B70142305105E8F02091FF01309177
S1131AC00002E0919102F0919202E40FF51F329727
S1131AD08081EDEBF0E08327880FF11DE80FF11D05
S1131AE0C895322F202D3196C895302530930002A9
S1131AF02093FF014F5F5F4F5093B7014093B601AE
S1131B0059C03E37D1F4109200021092FF01109296
S1131B10B7011092B60180917B029927FC01EE0F68
S1131B20FF1FEE0FFF1FE80FF91FE80FF91FE05822
S1131B30FD4F1282138211823BC080E28327E09121
S1131B409102F09192022091B6013091B701E20F17
S1131B50F31F80834091B6015091B7014230510583
S1131B60E8F02091FF0130910002E0919102F091A0
S1131B709202E40FF51F32978081EDEBF0E08327AA
S1131B80880FF11DE80FF11DC895322F202D3196D5
S1131B90C8953025309300022093FF014F5F5F4FBB
S1131BA05093B7014093B60183E08093A50202C02D
S1131BB01092A50281E090E00895CF93C1E020E067
S1131BC08FB7F894382F8091A602882391F58091DD
S1131BD0C102992781FF08C08CE792E09093240208
S1131BE08093230280E41AC082FF0FC0E091A50114
S1131BF0F091A601F0932402E093230282E48093FF
S1131C00A8018481992705960DC083FF12C08DEA2F
S1131C1091E090932402809323028FEF8093A80194
S1131C2081E090E09093B1018093B0012C2FC09398
S1131C30A6023FBF2223F1F08FB7F89499271092A0
S1131C404E0110924D0110926F0210926E028FBFDE
S1131C508EE70E943E0EC82F813061F08FB7F89452
S1131C60282F332788E08093A6022FBF83E59EE0C8
S1131C700E9455028C2F9927CF910895482F8FB732
S1131C80F894282F33279091760281E0809376028E
S1131C902FBF992319F080E090E008954CB95E9A23
S1131CA081E090E0089561E08FB7F894282F3327FE
S1131CB08091A602883019F460E06093A6022FBFD9
S1131CC08091A8019091C102803451F48FB7F894A7
S1131CD0282F332782E098279093C1022FBF17C083
S1131CE08FB7F894282F332784E098279093C10264
S1131CF02FBF8091A5019091A6010E94A40B8FB7DC
S1131D00F89499271092A6011092A5018FBF0E9402
S1131D10DD0D08958FB7F8949927209176021092DB
S1131D2076028FBF222309F4A4C08091A6028730D3
S1131D3031F41092A60283E59EE00E94550221E050
S1131D408091A60299278430910509F46EC08530EC
S1131D50910554F48230910561F1833091050CF0C2
S1131D6058C0019749F07CC08630910509F471C0D0
S1131D7006970CF463C074C082E08093A60220919D
S1131D804D0130914E018091A801EDEBF0E08327E5
S1131D90880FF11DE80FF11DC895322F202D3196C3
S1131DA0C895302530934E0120934D018091A801B0
S1131DB054C0E0912302F091240220916E023091EC
S1131DC06F02E20FF31F508180914D0190914E01FB
S1131DD0EDEBF0E0452F4927440FF11DE40FF11D11
S1131DE0C895982F802D3196C895902590934E01D3
S1131DF080934D012F5F3F4F30936F0220936E020B
S1131E008091B0019091B1012817390798F084E0CE
S1131E100FC08091AF0290E289270E943E0E282FC6
S1131E2080918E028093A6021BC050914D0185E0E3
S1131E308093A602852F0E943C0F11C080914D0112
S1131E4090914E01292F332786E08093A602822F9A
S1131E50F2CF87E08093A6028EE70E943E0E282FE1
S1131E60213039F088E08093A60283E59EE00E9449
S1131E70550281E090E00895982F8D57823078F4D0
S1131E808FB7F894282F33278091A60280938E026F
S1131E9083E08093A6029093AF022FBF9DE7892F22
S1131EA00E943E0E992708958FBF08958FB7F89426
S1131EB099270895E091A902F091AA023596248108
S1131EC02F5F248380910001909101018283938389
S1131ED03091940220FF06C08FB7F8949927D998BF
S1131EE0326005C08FB7F8949927D99A3D7F309313
S1131EF094028FBF84813091940281FF06C08FB712
S1131F00F8949927DA98316005C08FB7F894992727
S1131F10DA9A3E7F309394028FBF8181992787FD9F
S1131F2090958330910571F18430910534F48130BA
S1131F30910579F00297B1F02EC08730910541F1F7
S1131F40883091051CF40497C9F025C0089711F155
S1131F5022C08FB7F894282F3327D8988091940201
S1131F60846008C08FB7F894282F3327D89A8091BB
S1131F7094028B7F809394022FBF0DC08091B20195
S1131F808F5F03C08091B20181508093B20103C07E
S1131F90AA9A01C0AA981092AE0108958FB7F89436
S1131FA0682F7727E0917202F091730217A210A6AE
S1131FB084A195A19C01220F331F220F331F280FE8
S1131FC0391F4091550250915602CA01880F991F3A
S1131FD0840F951F280F391F53E0369527955A957E
S1131FE0E1F730935602209355026FBFCF010E9450
S1131FF0CA079C018FB7F89499272115310521F060
S11320003093730220937202E0917202F091730292
S113201014828FBF80EC8DB9B8980E944B07089545
S11320208FB7F8949927E0919502F091960217A240
S113203010A68FBF61E0CF010E94A40B8FB7F89464
S113204099271092A9018FBF08958F929F92AF9202
S1132050BF92DF92EF92FF920F931F93CF93DF9380
S113206081E0809374028091B4029091B502A091B2
S1132070B602B091B7020097A105B10509F484C076
S1132080DD240AE512E0EE24FF2461E070E00E2C6A
S113209002C0660F771F0A94E2F7CB01AA2797FDC7
S11320A0A095BA2F8090B4029090B502A090B60289
S11320B0B090B70288219921AA21BB210097A105DC
S11320C0B10509F457C080917F0299270196AA2788
S11320D097FDA095BA2FF801258136814781508557
S11320E0281B390B4A0B5B0B2583368347835087A8
S11320F02330310541055105ECF58081882369F4CD
S113210081819281A381B481280F391F4A1F5B1FEB
S1132110258336834783508713C0CB0180959095E0
S1132120AA2797FDA095BA2F88229922AA22BB221A
S11321308092B4029092B502A092B602B092B70215
S11321408091BE02813019F48FEF8093BE0290918A
S1132150BE029F5F9093BE028091EA018F5F8093DD
S1132160EA01E92FFF27E655FE4FD0828CE791E183
S11321700E945502D3940894E11CF11C075F1F4F81
S1132180F1E0FD1508F081CF0E94A701DF91CF9106
S11321901F910F91FF90EF90DF90BF90AF909F90B1
S11321A08F90089587B799278C7F009719F080E066
S11321B090E01AC06F9918C0379B03C088E090E084
S11321C013C087B7992783709070892B59F081B712
S11321D092B7891B803118F48CE190E005C088E146
S11321E090E002C080E190E0382F25B7237E8C3147
S11321F021F0883111F008C0000080B7992787705A
S11322009070892BC9F7237E232B25BF85B7806265
S113221085BF08950F931F93CF93DF939091A802E6
S113222086E0989F8001112400581D4FF801C48155
S1132230D58182819381059780F12081822F99270E
S11322408134910559F08234910524F48034910548
S113225021F11DC08234910571F019C081E090E034
S11322608AA39BA3F801818180937E0286E691E193
S11322700E94550204C081E090E08AA39BA3809150
S113228002018B83CE010E94CA07EC0106C0209391
S1132290AD0187E492E10E9455028FB7F894282F8C
S11322A03327209719F0F801C483D583F8011282EB
S11322B0138211828091A8028F5F81708093A8029B
S11322C02FBFDF91CF911F910F91089520917E022E
S11322D031E08FB7F8949091C10291FD06C09260ED
S11322E09093C10220937C0201C030E08FBF313053
S11322F011F40E94DD0D08951F93CF93DF93909105
S1132300EA01992319F482E090E015C08091A701B5
S1132310813019F48FEF8093A7018091A7018F5F1B
S11323208093A70191509093EA01E82FFF27E65587
S1132330FE4F80819927823008F0A5C0282F3327CB
S11323402115310521F02130310571F09CC08091B7
S11323505702909158029093AE028093AD0230934D
S11323605802209357028FC0E0917D02EE2309F4B6
S11323708AC08FB7F89499272091AF011091AC01CE
S11323808FBF33272230310521F02630310591F1FA
S113239072C08E2F9927880F991FFC01EF55FF4FAC
S11323A024913327D22FCC278E559F4FFC01849143
S11323B09927C82BD92B112309F05DC08FB7F89446
S11323C0282F332786E08093AF012FBFCE01AA27A1
S11323D0BB279C01AD0161E0862F0E945D07612F40
S11323E08BE00E94BA066FE3812F0E94BA060E9416
S11323F0CC0B49C0FF27E155FF4F8491C82FDD273F
S11324008FB7F894282F332782E08093AF012FBF32
S11324106BE380E00E94BA0680ED97E000000000C4
S113242000000000000000000000000001971816E2
S11324301906A4F369E380E00E94BA0688EC90E0F0
S11324400000000000000000000000000000000088
S1132450019718161906A4F3BB98BA980E942C0782
S113246080EC8DB9B8980E944B07CE01AA27BB27F0
S11324709C01AD0104C020E230E040E050E061E0A6
S1132480862F0E945D07DF91CF911F9108958FB72A
S1132490F894282F33278091C10288608093C10269
S11324A02FBF0E94DD0D0895629FD001739FF0013C
S11324B0829FE00DF11D649FE00DF11D929FF00DD0
S11324C0839FF00D749FF00D659FF00D9927729F07
S11324D0B00DE11DF91F639FB00DE11DF91FBD0192
S11324E0CF0111240895A1E21A2EAA1BBB1BFD01E2
S11324F00DC0AA1FBB1FEE1FFF1FA217B307E407DF
S1132500F50720F0A21BB30BE40BF50B661F771F36
S1132510881F991F1A9469F7609570958095909516
S10D25209B01AC01BD01CF01089539
S113252A010033008025009224200000201C0000B2
S113253A001900008016005D74140000C01200C562
S113254A4E110049121000BD04880552061C07E604
S113255A07B0087B09450A0F0BAA01F1013802806A
S10F256A02C7020E0355039C03E30301A7
S9030000FC
